:020000040000FA
:02000000FC28DA
:08000800A100030EA2000B1180
:100010009C0A20141C087F3C031D2D289C01A01461
:10002000AB0A2B08D73C031D1828AB019C032D28D5
:100030009D0A1D083C3C031D2D289D0120159E0A8C
:100040001E083C3C031D2D289E01A0159F0A1F0879
:10005000183C031D2D289F012016220E8300210825
:100060000900FC28A0101D0892001E0891001F081E
:1000700090003C200800FC281518F420151CF820DE
:100080001208872292000F396D209518F420951CD4
:10009000F820120E0F396D201108872291000F39B8
:1000A0006D201519F420151DF820110E0F396D2043
:1000B0009519F420951DF8201008872290000F391B
:1000C0006D20100E0F396D20061500000000000095
:1000D0000000000006110800FC2882077B28862803
:1000E00091289C28A728B228BD28C828D328DE2814
:1000F000E9280800FC28F820F820F820F820F8204B
:10010000F820F820F820F820F4207928F820F820AA
:10011000F820F820F820F820F820F820F420F82023
:100120007928F820F820F820F820F820F820F82086
:10013000F420F820F8207928F820F820F820F8207A
:10014000F820F820F420F820F820F8207928F8206A
:10015000F820F820F820F820F420F820F820F820E3
:10016000F8207928F820F820F820F820F420F8204A
:10017000F820F820F820F8207928F820F820F82036
:10018000F420F820F820F820F820F820F82079282A
:10019000F820F820F420F820F820F820F820F820A3
:1001A000F820F8207928F820F420F820F820F8200A
:1001B000F820F820F820F820F8207928F420F820FA
:1001C000F820F820F820F820F820F820F820F8206F
:1001D0007928F820F820F820F820F820F820F820D6
:1001E000F820F820F82079288614061486100800D4
:1001F00086140610861008008B018501860183167F
:10020000E0308500F03086008330810083120000EA
:1002100006158615000000000C3095000030900097
:1002200000309100003092009C019D019E019F01D1
:10023000A001A3019A019B01A401A0308B00A0188A
:10024000322069221A1859229A1859211A199A1912
:100250009A01241C38291D08003A031D38291E085C
:100260001706031D38291F081606031D38296222A8
:10027000A41C56291D08003A031D48291E0819060A
:10028000031D48291F081806031D482915140515C4
:100290001D08003A031D56291E082A06031D56296B
:1002A0001F082906031D56291510051100001F29D6
:1002B000FC281B146330920063309100633090007F
:1002C0001B183C201B1069221A18DA219A186D2974
:1002D0001A1970219A1912225A299A010800FC2829
:1002E0001B1415088C009501151500000D14A41899
:1002F0007C29151099019801A41815140D140030CB
:10030000920019089100180890000D183C208D01EA
:1003100069221A1C90290230A406013095060D149A
:100320009A1C9529A418B121A8291A1D9E290D14DB
:10033000990A19083C3C031DA72999019A1DA72970
:100340000D14980A1808183C031DA72998017C2948
:1003500015110C08A4181514150495009A0108002D
:10036000FC280D1415101908AA001808A90000305F
:1003700092002A089100290890000D183C208D0158
:1003800069229A1CC429D7291A1DCD290D14AA0A3D
:100390002A083C3C031DD629AA019A1DD6290D1412
:1003A000A90A2908183C031DD629A901B7299A01D1
:1003B0000800FC281B1415088C000D14151295104C
:1003C00095110030A8001E08A7001F08A6002808E5
:1003D000920027089100260890000D183C208D01FE
:1003E00069229A1CFA2928089D0027089E002608E1
:1003F0009F000D2A1A1D032A0D14A70A27083C3C4A
:10040000031D0C2AA7019A1D0C2A0D14A60A260802
:10041000183C031D0C2AA601E7290C0895009A0137
:100420000800FC281B1415088C0095019515000088
:100430000D14A4181E2A151097019601241895145E
:100440000030920017089100160890000D183C200B
:100450008D0169221A1C312A0130A406023095064A
:100460000D149A1C342A472A1A1D3D2A0D14970A86
:1004700017083C3C031D462A97019A1D462A0D1475
:10048000960A1608183C031D462A96011E2A951145
:100490000C08150495009A010800FC28201C4E2A1F
:1004A0002010A30A2308063C031D4E2AA3010800BE
:1004B000FC28051D5E2A15100511602A1514051566
:1004C0000800FC288515951001309322851108003D
:1004D000FC289A01061A712A1A144E22060E9A0551
:1004E000852A861A782A9A144E22060E9A05852A9B
:1004F000061B7F2A1A154E22060E9A05852A861B90
:10050000852A9A154E22060E9A050800FC289301AA
:10051000F63E031C8D2A930A882A0A3E930E930402
:1005200013080800FC280D08C6308C0000000000ED
:0C0530008C0B962A8D0B942A0800FC28E6
:084000000400010005000500A9
:02400E00F93F78
:00000001FF
